:03000000023B4D73
:0C3B4D0078FFE4F6D8FD758171023B940E
:1013F6000A53746172743A20004950436F6E6E65E9
:1014060063745245510A004950436F6E6E656374AA
:10141600003E432C562C43432CC0E4E0EFF2E5F0AB
:1014260020D1E8EDEAEEEC49500A003E432C4D414E
:10143600432C25303262583A25303262583A2530EC
:101446003262583A25303262583A25303262583A7A
:1014560025303262582C4D414320E0E4F0E5F10A94
:10146600003E432C5645522C20332E3120EEF220DE
:1014760025732025732CC2E5F0F1E8FF20495020A2
:10148600ECEEE4F3EBFF0A004A616E2032382032BC
:101496003030380030383A33393A3533003E432C51
:1014A6004C442C50524F473A202020202020202008
:1014B6002020202020202020202020202020202026
:1014C6002020202020202020202020202020202016
:1014D6002020202020202020202020202020202006
:1014E600202020202020202020202020202CC4E086
:1014F600F2E020EFF0EEF8E8E2EAE828F4E0E9EBC3
:10150600290A003E2A2C312CCEF1EDEEE2EDFBE568
:1015160020EFE0F0E0ECE5F2F0FB20F1E5F2E5E2A9
:10152600EEE3EE20E8EDF2E5F0F4E5E9F1E00A009D
:101536003E412C4130312C2562752E2562752E25B3
:1015460062752E2562752C495020E0E4F0E5F12005
:10155600E0E4E0EFF2E5F0E00A003E412C413032F3
:101566002C2562752E2562752E2562752E256275CF
:101576002C495020E0E4F0E5F120EEF1ED2E20F1CB
:10158600E5F0E2E5F0E00A003E412C4130332C253F
:1015960062752E2562752E2562752E2562752C497B
:1015A6005020E0E4F0E5F120F0E5E72E20F1E5F04B
:1015B600E2E5F0E00A003E412C4130342C2562750C
:1015C6002E2562752E2562752E2562752CCCE0F1CE
:1015D600EAE020F1E5F2E80A003E412C4130352CE4
:1015E6002562752E2562752E2562752E2562752C4F
:1015F600D8EBFEE70A003E532C4130362C256275A7
:101606002CC2F0E5ECFF20EEE6E8E42E20EAE2E864
:10161600F2E0EDF6E8E820282A3130ECF1290A005C
:101626003E2A2C312CC4EEEF2E20EFE0F0E0ECE564
:10163600F2F0FB20F1E5F2E5E2EEE3EE20E8EDF272
:10164600E5F0F4E5E9F1E00A003E422C5330312C96
:101656002562752CC6E4E0F2FC20E7E0EFF0EEF13F
:10166600E020F1EEE5E4E8EDE5EDE8FF20EEF2201E
:10167600F1E5F0E2E5F0E00A003E422C5330322C70
:101686002562752CCEE1ECE5ED20F120F1E5F0E2E6
:10169600E5F0EEEC20E1E5E720EAE2E8F2E0EDF63F
:1016A600E8E90A003E422C5330332C2562752CCFD4
:1016B600E5F0E5E7E0EFF3F1EA20EFF0E820EFEE02
:1016C600F2E5F0E520F1E2FFE7E820F120F1E5F0B0
:1016D600E2E5F0EEEC0A003E422C5330342C256253
:1016E600752CCDE5F220EFE5F0E5E4E0F7E820E43F
:1016F600E8E0E3EDEEF1F2E8EAE820E220F1E5F0D9
:10170600E2E5F00A003E422C5330352C2562752C5A
:10171600CAE0EDE0EB20F8E8F0EEEAEEE2E5F8E00C
:10172600F2E5EBFCEDEEE3EE20EEE1ECE5EDE00AB2
:10173600003E532C5330362C253032625825303239
:10174600625825303262582530326258253032626E
:101756005825303262582C4D414320E0E4F0E5F143
:1017660020F8E8F0EEEAEEE2E5F8E0F2E5EBFCED73
:10177600EEE3EE20EEE1ECE5EDE00A003E454E44F8
:101786000A0044756D70582020202020303020300B
:10179600312030322030332030342030352030367E
:1017A6002030372030382030392030412030422058
:1017B60030432030442030452030460A003A003A73
:1017C60020000A0044756D7044202020202030300F
:1017D6002030312030322030332030342030352054
:1017E6003036203037203038203039203041203014
:1017F600422030432030442030452030460A004500
:101806007272206B657900526420656570726F6D27
:101816000A005264204D454D0A00526420436F640D
:10182600650A0044656275674950204F4E0A0044B8
:10183600656275674950204F46460A0044656275E1
:101846006755736572204F6E0A0044656275675569
:10185600736572204F46460A0044656275674D738C
:1018660067204F6E0A0044656275674D7367204FA7
:1018760046460A00436F6E666967206C6F636B218C
:101886000A00577220656570726F6D0A00205361F9
:10189600766520656570726F6D210A00457272204B
:1018A6004D414321004C6F61643E3E002A003C419D
:1018B60030313D003C4130323D003C4130333D004B
:1018C6003C4130343D003C4130353D003C413036F2
:1018D6003D003C21003C5330313D003C5330323D0D
:1018E600003C5330333D003C5330343D003C5330D4
:0918F600353D003C5330363D0045
:0644A700010B00010900F9
:10446600C2AFC28E438910758BFF758DB7D2ABD2A2
:044476008ED2AF2211
:03001B00023A2383
:103A2300C0E0C083C082C0D0C2AFC28E758BFF75A9
:103A33008DB720060675A61E75A6E10509D202E517
:103A43000B6002050BE50AD394014002150A050E2B
:103A5300E50E540F7050D20EE50E543F701AD2008B
:103A6300907B01E0601204F0E0D394B4400A9080AC
:103A7300007480F0C2AF80FE907AFCE0600204F034
:103A8300907578E0600214F0907B02E0D3940140DB
:103A930003E014F0300502050CE50DD394644004F3
:103AA300D2068002050DE508D3940140021508D221
:0C3AB3008ED2AFD0D0D082D083D0E032D1
:1008A400C291C290D2B5C20B7D027C007F07124375
:1008B400FA8F25E525646060097D017F601243B2EB
:1008C400D20BE4FDFC7F0B1243FA8F25E52530E6BD
:1008D400097D04E4FF1243D6D20B7D017C007F071F
:1008E4001243FA8F25E5257008FD7FFF1243B2D22B
:1008F4000B300B03126000C2AFC288C2A8C2AA7533
:100904008900123DE29077B5E0B4FA09A3E064CE21
:1009140070030209A4E4F52574AD2525F582E434B9
:1009240077F583E4F00525E525B443EC9077B574B9
:10093400FAF0A374CEF0A374CCF09077BB740AF0F1
:10094400E4A3F0A304F0A3F09077C07403F0A374BD
:10095400CCF09077B174FFF0A3F0A3F0E4A3F0908F
:1009640077CC7405F0E4F525E5252401FFE433FE96
:1009740074AD2525F582E43477F583E0FD12444D0A
:100984000525E525C3944340DFE4F5A775A61E7548
:10099400A6E1907FF0F0A3F09080007480F080FED8
:1009A400D2AF9077C07403F0A374CCF0E49077BF17
:1009B400F0123688C2B51228B2C20612413B9077B3
:1009C400CCE0C3940350037403F0D20BC20DC20CE9
:1009D400D293200B077E137FF61232A3E49079ECB6
:1009E400F0124466C2AFA37408F090772B7424F01D
:1009F400E4A3F09077B5E090772DF09077B6E0908F
:100A0400772EF09077B7E090772FF09077B8E0905A
:100A14007730F09077B9E0907731F09077BAE09042
:100A24007732F0750A01E49079EEF0C207C208C289
:100A340009C20AD2AF75A70775A61E75A6E11243AF
:100A44008B200B19AF257E007D031233A4E4FF1223
:100A540038387E777FECE4FB7D01123594907B017E
:100A6400E060037401F0E4907578F0A37455F0A38A
:100A74007481F0E4F50CE4F50D907578E0700312E0
:100A84001F22907B02E0B401119080007410F0E406
:100A9400907B02F0D20BC20CC20D908008E0F525C9
:100AA40030E405D2077410F0E52530E508D209904A
:100AB40080087420F0E52530E608D2089080087498
:100AC40040F0E50CD394034023908002E4F090803E
:100AD40001F0908000F0E50CD39406400FE4F50C8F
:100AE400C2039079EEF0750A0112413B9080A0E0B8
:100AF4007003123E609080B8E07003123EDA90807A
:100B0400D0E07003123FB9908000E07013300710FA
:100B140012319F9077A8EFF0D3940040031200267F
:100B2400908002E07006908000E06005D205020A21
:100B34007AC205E4F50C907578E06003020A7A3015
:100B44000912122DA89077A8EFF0D394004005E085
:100B5400FF12447A200803020CD9122C339077A890
:100B6400EFF07003020A7A9077ECE054BF247F70B0
:100B740003020C3C147003020C1424026003020CE4
:100B84006F200B077E137FFF1232A3300F792003EF
:100B9400769077C4E070069077C8E0605B907AF84E
:100BA400E0FF9077C4E0B50724907AF9E0FE9077EF
:100BB400C5E0B50618907AFAE0FE9077C6E0B5066F
:100BC4000C907AFBE0FE9077C7E06E602B9077C8BC
:100BD400E06F7033907AF9E0FF9077C9E0B50727AA
:100BE400907AFAE0FF9077CAE0B5071B907AFBE0B1
:100BF400FF9077CBE0B5070F9079EE7401F0120007
:100C040021750A01020CD9907AF874FFF0020CD90C
:100C1400907B01E060037401F0907AF0E0FF90773C
:100C2400EEE06F6003020CD9907AF0E004F0E4F592
:100C34000A9079ECF0020CD9300303020CD99077B6
:100C4400BBE07003020A7A1244AED203E4F50A90C0
:100C540079ECF0907AFC04F0E4907AEFF0A3F020C1
:100C64000B737E147F0D1232A3806A907B01E060C7
:100C7400037401F03003529077ECE020E74B907757
:100C8400EEE0FF907AEFE0FE6F600D907AF7E0708F
:100C940007EE146F703F8013907AEFE004F09077C2
:100CA400A8E0FFD394044003124222907474748227
:100CB400F0A37401F09077EEE0907476F07E747F88
:100CC400747D03123D62020A7A300F0920030690F4
:100CD4007AF874FFF0200303020D8EE50A706B129C
:100CE40042D3EF60207E787FEC9078EDE02404FD21
:100CF400123D62907AF7E06003020A7A9077CCE0C2
:100D0400F50A020A7A907AFCE0D3943C403C907A4B
:100D1400F7E07036907AFC04F090772AE0702B129A
:100D24004494E49078ECF0A37412F0907AF0E0909C
:100D340078EEF0A374FDF090757B63A2019078F0D7
:100D440063A2017F121227A4809B124489EF6015CD
:100D54009074747483F0E4A3F07E747F747D021243
:100D64003D62020A7AE50A64016003020A7A907914
:100D7400ECE004F0E0C394055003020CE9C203E480
:100D84009079EEF0120021020A7AE50A6401600308
:100D9400020A7A9079EEE014604624FE60421470F0
:100DA40003020E7C24046003020A7AE4F50C200F8B
:100DB400139079EE7404F09079ECE05401F0750A24
:100DC40001020A7A9080027410F0E49079EEF090B7
:100DD40079EC04F0750AC8907AF874FFF0020A7A84
:100DE400907AF8E07003020E6B9078EC7480F090C7
:100DF40078EE7401F0E4A3F0A304F0A37430F0A33C
:100E0400747BF0E4F52574F32525F582E43478F554
:100E140083747DF074F42525F582E43478F583E455
:100E2400F0E52524079078EDF07C7A7DF89077C082
:100E3400E0FAA3E0FB7F02123C5E7E787FECE525BE
:100E44002409FD123D62907AF7E0601B1244AED291
:100E540003E4F50A9079ECF0907AFC04F0E4907ADB
:100E6400EFF0A3F0020A7A9079EE7404F09077CC54
:100E7400E02432F50A020A7A9080027410F0750AAE
:100E8400039079ECE06401FFF09079EE7401F0EFE7
:100E940070199077C8E06013FCA3E0FDA3E0FEA303
:100EA400E0FF907AF81222EA020A7A9077C4E0FC12
:100EB400A3E0FDA3E0FEA3E0FF907AF81222EA0289
:040EC4000A7A80FE28
:010EC8002207
:100026009077EDE0B444047F0180027F009077EC86
:10003600E0B447047E0180027E00EE5F604A90775E
:10004600B5E09077EEF09077B6E09077EFF09077A6
:10005600B7E09077F0F09077B8E09077F1F090778E
:10006600B9E09077F2F09077BAE09077F3F0907776
:10007600ED7452F090772463A2019080A863A201E8
:100086007F061227A402089A9077A8E0C394085026
:10009600030208A39077B5E0FF9077EEE06F600368
:1000A6000208A39077B6E0FF9077EFE06F60030257
:1000B60008A39077B7E0FF9077F0E06F600302083F
:1000C600A39077B8E0FF9077F1E06F60030208A392
:1000D6009077B9E0FF9077F2E06F60030208A39093
:1000E60077BAE0FF9077F3E06F60030208A390779A
:1000F600EDE0B44415907724E0B4FF0E63A20190BE
:1001060080A863A2017F061227A4907B01E060030A
:100116007401F0907B027464F09077ED7452F09065
:1001260077ECE0646D60030202A37BFF7A14791713
:100136001219617BFF7A1479319077B5E0F52EA319
:10014600E0F52FA3E0F530A3E0F531A3E0F532A307
:10015600E0F533121961752EFF752F1475308E7503
:1001660031FF75321475339A7BFF7A147967121949
:10017600617BFF7A1479A31219617BFF7A157909DD
:100186001219617BFF7A1579369077BBE0F52EA3BD
:10019600E0F52FA3E0F530A3E0F5311219617BFFFE
:1001A6007A1579609077C4E0F52EA3E0F52FA3E0E9
:1001B600F530A3E0F5311219617BFF7A15798E903F
:1001C60077C8E0F52EA3E0F52FA3E0F530A3E0F520
:1001D600311219617BFF7A1579BC9077B1E0F52E63
:1001E600A3E0F52FA3E0F530A3E0F5311219617B0A
:1001F600FF7A1579DF9077ADE0F52EA3E0F52FA312
:10020600E0F530A3E0F5311219617BFF7A1579FC30
:100216009077CCE0F52E1219617BFF7A16792612BB
:1002260019617BFF7A16794FA20FE433F52E121966
:10023600617BFF7A16797F907AF7E0F52E121961C5
:100246007BFF7A1679AA907B01E0F52E1219617B65
:10025600FF7A1679DD90772AE0F52E1219617BFF79
:100266007A17790BA201E433F52E1219617BFF7A16
:10027600177937907AF1E0F52EA3E0F52FA3E0F594
:1002860030A3E0F531A3E0F532A3E0F533121961AE
:1002960012349E7BFF7A177982121961229077ECCD
:1002A600E0644C70757E177F881232A39077F4E075
:1002B600F526A3E0F527E4F5297E177FC31232A3BE
:1002C6007D03AF27AE261233A47E177FC51232A355
:1002D600E4F528852782852683E0FF74F62528F530
:1002E60082E43477F583EFF00527E52770020526CB
:1002F6000528E528B410DC7E777FF6E4FB7D101236
:1003060035947E177FC81232A30529E529C39410B8
:1003160040A77E177FC81232A3229077ECE0646C68
:10032600705CF52A7E177FCA1232A3E4F529AF2A3C
:100336007E007D031233A47E177FC51232A3E4F537
:1003460028A82AE6FF74F62528F582E43477F58393
:10035600EFF0052A0528E528B410E67E777FF6E457
:10036600FB7D101235947E177FC81232A30529E54E
:1003760029C3940840B87E177FC81232A32290770B
:10038600ECE0644B7061F52874DE2528F582E434D0
:1003960077F583E0603274DE2528F582E43477F55C
:1003A60083E0F4602374DE2528F582E43477F58350
:1003B600E0FF74F42528F582E43477F583E0B50789
:1003C600100528E528B408C09075787432F0020844
:1003D6009A9077EC7421F0300B0302089A7E187F0E
:1003E600051232A302089A9077ECE0B4521A200B59
:1003F600077E187F0D1232A39077EC7472F07E7729
:100406007FEC7D08123CE2229077ECE0644970456F
:10041600200B077E187F181232A39077F4E0F5269A
:10042600A3E0F527E4F528852782852683E0FF7477
:10043600F62528F582E43477F583EFF00527E527DE
:10044600700205260528E528B480DC7E777FEC7DE2
:100456008A123CE2229077ECE064437079A3E06470
:10046600527046200B077E187F201232A39077F435
:10047600E0F526A3E0F527E4F5288527828526837F
:10048600E493FF74F62528F582E43477F583EFF0DC
:100496000527E527700205260528E528B480DB7EBA
:1004A600777FEC7D8A123CE2229077EDE06457601C
:1004B600030208A39077F4E0F526A3E0F52774F687
:1004C6002528F582E43477AD82FC7B80AF27AE2603
:1004D60012429F02089A9077ECE06444600302059A
:1004E6006D9077F4E0FF6444700302089AEFB4312C
:1004F6000CC20B7E187F291232A302089A9077F459
:10050600E0B4300CD20B7E187F351232A302089A63
:100516009077F4E0B4320CD20C7E187F421232A3EC
:1005260002089A9077F4E0B4330CC20C7E187F5020
:100536001232A302089A9077F4E0B4340CD20D7EFE
:10054600187F5F1232A302089A9077F4E0B4350C54
:10055600C20D7E187F6C1232A302089A9077F4E0DF
:10056600FF12001E02089A907578E07013200B07A0
:100576007E187F7A1232A39077EC7421F002089AE3
:100586009075787432F09077ECE0FFB4510A908061
:10059600007480F0C2AF80FEEF64577045200B07F1
:1005A6007E187F881232A39077F5E09077A8F0E462
:1005B600F5289077A8E0FFE528C39F400302089A34
:1005C60074F62528F582E43477F583E0FF9077F416
:1005D600E025282423F582E43476F583EFF0052818
:1005E60080D09077ECE06453600302069C200B07F2
:1005F6007E187F931232A39077B5E0FF90762CE0B9
:100606006F703C9077B6E0FF90762DE06F7030907B
:1006160077B7E0FF90762EE0B507249077B8E0FF35
:1006260090762FE0B507189077B9E0FF907630E026
:10063600B5070C9077BAE0FF907631E06F601690C0
:1006460077EC7421F0300B0302089A7E187FA21211
:1006560032A302089AE4F528E4F50DAF28FE7423C8
:100666002528F582E43476F583E0FD12444D05280D
:10067600E528C394FE40E19080007480F0C2AFE4A8
:10068600907FF0F0A3F0907FFD74AAF0A374FFF0C2
:10069600A37455F080FE9077ECE0644F704C907731
:1006A600F4E0F526A3E0F527E5274526700A200B9A
:1006B600077E187FAB1232A3200B077E187FB2127B
:1006C60032A3E4F52874F62528F582E43477F58319
:1006D600E0852782852683F00527E5277002052613
:1006E6000528E528B480DE02089A9077ECE0FFB48E
:1006F60045279080007480F09077F4E0FDA3E090A9
:100706007FF0CDF0A3EDF0C2AF907FFD74AAF0A309
:1007160074FFF0A37455F080FEEF64656003020871
:100726009A9077F4E0FFA3E0907FF0CFF0A3EFF08C
:10073600E4F526F527D3907FF1E09527907FF0E04A
:1007460095264020E4F50D2527FFE5263401FE8594
:100756002782852683E0FD12444D0527E527700292
:10076600052680D17E187FB4123BD9EF4E60201249
:1007760000039077BBEFF01200039077BCEFF01206
:1007860000039077BDEFF01200039077BEEFF07E86
:10079600187FBA123BD9EF4E60201200039077C43F
:1007A600EFF01200039077C5EFF01200039077C6C2
:1007B600EFF01200039077C7EFF07E187FC0123B70
:1007C600D9EF4E60201200039077C8EFF0120003B5
:1007D6009077C9EFF01200039077CAEFF01200038A
:1007E6009077CBEFF07E187FC6123BD9EF4E602094
:1007F6001200039077B1EFF01200039077B2EFF09A
:100806001200039077B3EFF01200039077B4EFF085
:100816007E187FCC123BD9EF4E60201200039077F2
:10082600ADEFF01200039077AEEFF0120003907771
:10083600AFEFF01200039077B0EFF07E187FD21280
:100846003BD9EF4E60081240DE9077CCEFF0E4F52E
:1008560028E4F50DE5282401FFE433FE74AD2528D0
:10086600F582E43477F583E0FD12444D0528E5284A
:10087600C3944340DC9080007480F0C2AFE4907F64
:10088600F0F0A3F0907FFD74AAF0A374FFF0A374B8
:0D08960055F080FE7E777FEC7D08123CE27D
:0108A3002232
:10426700AE07EEC39430400BEED394395005EE24DD
:10427700D0FF22EEC39461400BEED394665005EE57
:1042870024A9FF22EEC39441400BEED39446500578
:08429700EE24C9FF22AF06224C
:10443300907723E004F07006907722E004F0907701
:0A44430022E0FEA3E0FF124417225E
:10000300124433124267EFC454F0FEC00612443365
:08001300124267D0E02FFF222A
:1040DE00E4907C43F0124433907C44EFF0C3943070
:1040EE004018E0FFD394395011907C43E0247BF5C7
:1040FE0082E43475F583EFF08011907C43E0247BED
:10410E00F582E43475F583E4F0800C907C43E00492
:10411E00F0E0D3940840BE752E00752F0075300068
:0C412E00E4F5317B017A75797B122A8F51
:01413A002262
:043BD9008E2B8F2C74
:103BDD00907722E4F0A374FFF0124433EF606EF49B
:103BED00606B852C82852B83E493B507EC752D01D5
:103BFD00E52C252DF582E4352BF583E49360259096
:103C0D007723E0252DFF907722E03400FE12441734
:103C1D00E52C252DF582E4352BF583E493B50704CA
:103C2D00052D80CCE52C252DF582E4352BF583E48F
:103C3D009370A6E52D24FFFFE434FFFE907723E07B
:103C4D002FF0907722E03EF07E007F0122E4FEFF10
:013C5D002244
:103688007E187FD8123BD9EF4E70037F01227E1837
:103698007FDB123BD9EF4E600C124433EF24D02469
:1036A800FF920F8002D20F7E187FE1123BD9EF4EB6
:1036B800600C124433EF24D0907AF7F08005E49040
:1036C8007AF7F07E187FE7123BD9EF4E600C124470
:1036D80033EF24D0907B01F08005E4907B01F07EED
:1036E800187FED123BD9EF4E600C124433EF24D013
:1036F80090772AF08005E490772AF07E187FF312FD
:103708003BD9EF4E600C124433EF24D024FF9201D2
:103718008002C2019077B563A201907AF163A20199
:103728007F061227A430013B7E187FF9123BD9EFA0
:103738004E6030120003907AF1EFF0120003907A95
:10374800F2EFF0120003907AF3EFF0120003907A90
:10375800F4EFF0120003907AF5EFF0120003907A7C
:06376800F6EFF07F0022E5
:104194009079EDE0C3947C503D9079EDE0FE04F01D
:1041A400742B2EF582E43477F583EFF0BF0A279061
:1041B40079EDE0FF04F0742B2FF582E43477F58376
:1041C400E4F09079EDE0FF1239839079ED7408F012
:0741D40090772CE004F022BB
:10413B009080007480F09077AD63A201F583F582D7
:10414B0063A2017F081227A49077B563A201908028
:10415B008863A2017F0A1227A4908092E4F0A374D3
:10416B0032F0A37401F09077BFE0FF9080B1F09034
:10417B0080E1EFF09080957455F0A3F0908000747F
:09418B0001F090800974F0F022AB
:103E6000908009E04410F09080A0E0706C9080A1F8
:103E70007482F09080A874FFF0A3F0A3F0A3F07F09
:103E8000039080AEEFF07FCBA3EFF07F039080AC88
:103E9000EFF0A374CBF09080007402F0907C3512A8
:103EA00022F600000000907C35E0908040F0907C8D
:103EB00036E0908041F0907C37E0908042F0907C3A
:103EC00038E0908043F0A3E4F0A3F0A3F0A3F090D7
:093ED0008018F0A3F0A3F0A3F0A8
:013ED90022C6
:103FB900908009E04440F09080D17482F09077C0FD
:103FC900E0FF9080DEF09077C1E0FF9080DFF09015
:103FD90080027402F0907C391222F60000000090F1
:103FE9007C39E0908058F0907C3AE0908059F090CC
:103FF9007C3BE090805AF0907C3CE090805BF0A3A1
:10400900E4F0A3F0A3F0A3F0908030F0A3F0A3F0C4
:02401900A3F012
:01401B002282
:103EDA00908009E04420F09080B8E0706C9080B93E
:103EEA007482F07F039080C6EFF07FCDA3EFF07F5E
:103EFA00039080C4EFF0A374CDF09080C074FFF0FB
:103F0A00A3F0A3F0A3F09080017402F0907C3D121C
:103F1A0022F600000000907C3DE090804CF0907CFE
:103F2A003EE090804DF0907C3FE090804EF0907C97
:103F3A0040E090804FF0A3E4F0A3F0A3F0A3F09048
:093F4A008024F0A3F0A3F0A3F021
:013F5300224B
:103C5E008C268D27A907EAFDE975F018A424ACFF80
:103C6E00E5F034808F82F583EDF0EBFDE975F01809
:103C7E00A4FFAEF024ACFBEE34808B82F583A3ED73
:103C8E00F08527828C83E0FDEF24A8FFEE3480FEC2
:103C9E008F82F583EDF08527828C83A3E08F828E51
:103CAE0083A3F0852782852683A3A3E0FDE975F023
:103CBE0018A424A8FFE5F03480FE8F82F583A3A319
:103CCE00EDF08527828C83A3A3A3E08F828E83A33E
:043CDE00A3A3F0228A
:063CE2008D2BAB07AA06C2
:103CE800908000E020E572907C35E0FCA3E0FDA325
:103CF800E0FEA3E0F52F8E2E8D2D8C2CAE02AF03A7
:103D08008E838F8263A201E52E540744C0F5838514
:103D18002F8263A201AF2B122816E4FCFDFEE52FCB
:103D2800252BF52FEE352EF52EED352DF52DEC3511
:103D38002CF52C908040E52CF0A3E52DF0A3E52E82
:103D4800F0A3E52FF09080007420F0AF2FAE2EADD9
:093D58002DAC2C907C351222EAFE
:013D6100223F
:063D62008D26AB07AA0646
:103D6800908002E020E572907C39E0FCA3E0FDA39E
:103D7800E0FEA3E0F52A8E298D288C27AE02AF033A
:103D88008E838F8263A201E529540744D0F5838589
:103D98002A8263A201AF26122816E4FCFDFEE52A5A
:103DA8002526F52AEE3529F529ED3528F528EC35AF
:103DB80027F527908058E527F0A3E528F0A3E52903
:103DC800F0A3E52AF09080027420F0AF2AAE29AD66
:093DD80028AC27907C391222EA84
:013DE10022BF
:023838008F27D8
:10383A00908001E030E5037F0022907C3DE0FCA30C
:10384A00E0FDA3E0FEA3E0F52B8E2A8D298C2890BB
:10385A007AF163A201E52A540744C8F583852B82CD
:10386A0063A2017F0612282CE52B2406F52BE435EA
:10387A002AF52AE43529F529E43528F5289079EF3F
:10388A0063A201E52A540744C8F583852B8263A203
:10389A0001AF2712282CE4FCFDFEE52B2527F52B8A
:1038AA00EE352AF52AED3529F529EC3528F5289043
:1038BA00804CE528F0A3E529F0A3E52AF0A3E52B3F
:1038CA00F09080017420F0AF2BAE2AAD29AC28907D
:0738DA007C3D1222EAAF273A
:0138E10022C4
:10319F009081E0E0F526052605260526052605265D
:1031AF0005260526052605260526908010E0F5291B
:1031BF00A3E0F52AA3E0F52BA3E0F52C9081E1E045
:1031CF00F5260526052605260526052605260526A8
:1031DF00052605260526908014E0F52DA3E0F52E93
:1031EF00A3E0F52FA3E0F530E52FB52B08E530B5BB
:1031FF002C037F0022E4F526E52F540744E0F583E6
:10320F0085308263A2019077EC63A2017F081228B8
:10321F005C9077EE63A20190772463A2017F061280
:10322F0027A49077ECE0F527A3E0F528E4F52690A6
:10323F0077ECE0702AA3E024F8F526E52F54074435
:10324F00E0F58385308274082582F582E43583F5B5
:10325F008363A2019077EC63A201AF2612285CAEC4
:10326F0027E4FCFDE5302528F530E52F3EF52FED61
:10327F00352EF52EEC352DF52D908014E52DF0A380
:10328F00E52EF0A3E52FF0A3E530F0908000744019
:03329F00F0AF2667
:0132A2002209
:102C33009081E6E0F52605260526052605260526C8
:102C430005260526052605260526908028E0F52974
:102C5300A3E0F52AA3E0F52BA3E0F52C9081E7E0B0
:102C6300F526052605260526052605260526052619
:102C730005260526052690802CE0F52DA3E0F52EEC
:102C8300A3E0F52FA3E0F530E4F526E52FB52B0AF5
:102C9300E530B52C05C208022D8DE52F540744F00D
:102CA300F58385308263A2019077EC63A2017F08EC
:102CB30012285C9077ECE0F527A3E0F528E528459A
:102CC3002770099080027410F07F0022907AF8E058
:102CD300FFF4602D9077EEE06F7076907AF9E0FF65
:102CE3009077EFE06F706A907AFAE0FF9077F0E008
:102CF3006F705E907AFBE0FF9077F1E06F60228067
:102D0300509077EEE0907AF8F09077EFE0907AF9D0
:102D1300F09077F0E0907AFAF09077F1E0907AFB18
:102D2300F09077ECE0702AA3E024F8F526E52F5421
:102D33000744F0F58385308274082582F582E435F3
:102D430083F58363A2019077EC63A201AF26122877
:102D53005CAE27E4FCFDE5302528F530E52F3EF594
:102D63002FED352EF52EEC352DF52DAF2CAE2BADED
:102D73002AAC29AB30AA2FA92EA82DD31222D940D1
:102D8300099080027410F07F002290802CE52DF0D2
:102D9300A3E52EF0A3E52FF0A3E530F090800274B5
:042DA30040F0AF2627
:012DA7002209
:102DA8009081E3E0F5260526052605260526052655
:102DB8000526052605260526052690801CE0F5290A
:102DC800A3E0F52AA3E0F52BA3E0F52C9081E4E03D
:102DD800F5260526052605260526052605260526A3
:102DE800052605260526908020E0F52DA3E0F52E82
:102DF800A3E0F52FA3E0F530E4F526E52FB52B0A7F
:102E0800E530B52C05C209022EF3E52F540744E836
:102E1800F58385308263A20190747863A2017F0EE6
:102E2800122872907478E0F527A3E0F52890748052
:102E3800E0FFF46045907AF1E0FEEF6E706EA3E07B
:102E4800FF907481E06F7064907AF3E0FF90748271
:102E5800E06F7058907AF4E0FF907483E06F704CE4
:102E6800907AF5E0FF907484E06F7040907AF6E015
:102E7800FF907485E06F60048032D2D9907478E056
:102E8800702AA3E024F2F526E52F540744E8F583D9
:102E9800853082740E2582F582E43583F58363A23A
:102EA8000190747863A201AF26122872AE27E4FC61
:102EB800FDE5302528F530E52F3EF52FED352EF5CB
:102EC8002EEC352DF52DAF2CAE2BAD2AAC29AB3021
:102ED800AA2FA92EA82DD31222D95006E5284527B6
:102EE80070099080017410F07F0022908020E52DF9
:102EF800F0A3E52EF0A3E52FF0A3E530F0908001D4
:052F08007440F0AF264B
:012F0D0022A1
:0432A3008E2B8F2CB3
:1032A700E4F52DF52E908000E030E511052EE52E92
:1032B7007002052DD394E8E52D940340E890800033
:1032C700E030E5030233A3907C35E0FCA3E0FDA3E7
:1032D700E0FEA3E0F5328E318D308C2FE532FFE52D
:1032E700315407FEE42FF52EEE34C0F52D852E82DE
:1032F700F5837423F0052EE52E7002052D532DC797
:10330700F582852D83740AF0052EE52E7002052DB2
:10331700532DC79077B563A201852D83852E8263D0
:10332700A2017F061228167406252EF52EE4352DE8
:10333700F52D852B83852C8263A201852D83852E10
:103347008263A2011227FAE4FCFDFE907C35E0F8C7
:10335700A3E0F9A3E0FAA3E02FFFEE3AFEED39FD73
:10336700EC38FCEF2408FFE43EFEE43DFDE43CFCC2
:10337700907C351222EA907C35E0908040F0907C7A
:1033870036E0908041F0907C37E0908042F0907C6E
:0C33970038E0908043F09080007420F03B
:0133A3002207
:063594008E2B8F2C8D2D03
:10359A00E4F52EF52F908000E030E511052FE52F98
:1035AA007002052ED394E8E52E940340E89080003B
:1035BA00E030E503023687907C35E0FCA3E0FDA30A
:1035CA00E0FEA3E0F5338E328D318C30E533FFE532
:1035DA00325407FEE42FF52FEE34C0F52E852F82E4
:1035EA00F5837423F0052FE52F7002052E532EC79D
:1035FA00F582852E83EBF0052FE52F7002052E53F9
:10360A002EC79077B563A201852E83852F8263A288
:10361A00017F061228167406252FF52FE4352EF59C
:10362A002E852B83852C8263A201852E83852F828A
:10363A0063A201AF2D1228167408252DF52DFFE47B
:10364A00FCFDFEE5332FF533EE3532F532ED35313B
:10365A00F531EC3530F530908040E530F0A3E531B6
:10366A00F0A3E532F0A3E533F09080007420F0AFC8
:0D367A0033AE32AD31AC30907C351222EA17
:013687002220
:023983008F3F74
:10398500E4F540F541908000E030E5110541E54161
:1039950070020540D394E8E540940340E890800028
:1039A500E020E579907C35E0FCA3E0FDA3E0FEA3F3
:1039B500E0F5458E448D438C42E545FFE5445407CB
:1039C500FEE42FF541EE34C0F54090772B63A2015C
:1039D50085408385418263A201AF3F122816E4FC2E
:1039E500FDFEE545253FF545EE3544F544ED35430A
:1039F500F543EC3542F542908040E542F0A3E543BE
:103A0500F0A3E544F0A3E545F09080007420F0AF05
:0D3A150045AE44AD43AC42907C351222EA30
:013A22002281
:0633A4008E2B8F2CAB05FF
:1033AA00E4F52DF52E908000E030E511052EE52E8E
:1033BA007002052DD394E8E52D940340E89080002F
:1033CA00E030E50302349D907C35E0FCA3E0FDA3E8
:1033DA00E0FEA3E0F5328E318D308C2FE532FFE529
:1033EA00315407FEE42FF52EEE34C0F52D852E82DA
:1033FA00F5837423F0052EE52E7002052D532DC793
:10340A00F582852D83EBF0052EE52E7002052D90B1
:10341A0077B563A201852D83852E8263A2017F067B
:10342A001228167406252EF52EE4352DF52D532D6A
:10343A00C7E52B852E82852D83F0052EE52E700299
:10344A00052D532DC7F582852D83E52CF0052EE534
:10345A002E7002052D532DC7E532240AF532E435C4
:10346A0031F531E43530F530E4352FF52F908040D1
:10347A00E52FF0A3E530F0A3E531F0A3E532F090B3
:10348A0080007420F0AF32AE31AD30AC2F907C3575
:03349A001222EA11
:01349D00220C
:10441700E5D220E0FBC2AF438E2075D2028F828E99
:0B44270083E0FFE4F5D2538EDFD2AF3C
:014432002267
:10444D00E5D220E0FBC2AF43D2028F828E83EDF026
:09445D0075D25063D250D2AF2297
:103DE200E4FDED2401FFE433FE12441774AD2DF51A
:103DF20082E43477F583EFF00DBD3FE6E4FDED2478
:103E02007FFFE433FE12441774A32DF582E4347568
:103E1200F583EFF074A32DF582E43475F583E07039
:103E22001B74A32DF582E43475F5837420F074A419
:103E32002DF582E43475F583E4F080040DBD80BE77
:103E4200E4907622F0FDEDFF7E0012441774232DDC
:0D3E5200F582E43476F583EFF00DBDFEE956
:013E5F002240
:02429F008B2B67
:1042A100A2AF9210C2AF85A22C53A2FE8E838F8241
:1042B10005A28C838D8274091228A0E52B53A2FEDE
:1042C10043A2201228A253A2DF852CA2A21092AFF2
:0142D100FFED
:0142D20022C9
:1043FA00A2AF9210C2AF8C838D82EF1228A043A283
:0C440A00201228A253A2DFA21092AFFFE4
:014416002283
:0243B2008F2654
:1043B400A2AF9210C2AFE4F5838D8274061228A0D6
:1043C400E52643A2201228A253A2DFA21092AF7FB7
:0143D40001E7
:0143D50022C5
:0243D6008F2630
:1043D800A2AF9210C2AFE4F5838D82740A1228A0AE
:1043E800E52643A2201228A253A2DFA21092AF7F93
:0143F80001C3
:0143F90022A1
:1026C900A907E7FFA805EF93C3966008403B74FC90
:1026D9002FFF80F00F08EF93C3966008402B74FB1F
:1026E9002FFF80E00F08EF93C3966008401B74FA30
:1026F9002FFF80D00F08EF93D3966008400B74F931
:102709002FFF80C01F1F1F1F1FEF54FEF80303F781
:10271900E893FC08E893FD08E893FE08E893FF2294
:1027290009E993C39D6008402974FB29F980F109DF
:10273900E993C39E6008401A74FA29F980E209E90D
:1027490093D39F6008400B74F929F980D31919199B
:102759001919E9C313C313FF22740093F8ECC39842
:102769004024701F740193F8EDC3984019701474D4
:0E2779000293F8EEC398400E7009740393F8B3
:10278700EFC39840037F00227F0122EDF8E6F008AF
:10279700A3DFFA22EDF8E0F608A3DFFA22E0A3634D
:1027A700A201F0A363A201DFF475A2002263A201D4
:1027B700F0A363A20122E0A363A201F0A363A20135
:1027C700E0A363A201F0A363A201E463A201F0A363
:1027D70063A201DFE175A20022E0A363A2016DFEFF
:1027E700936CFDEE058393FC158363A201DFEA7505
:1027F700A200227F00E493A363A201F00F600CA361
:10280700E583C2E3F58363A20180EA75A20022E0B3
:10281700A363A201F0A3E583C2E3F58363A201DF0B
:10282700EE75A20022E0A363A201F0A3E583C2E450
:10283700D2E3F58363A201DFEC75A20022E0A36374
:10284700A201F0A3E58344F8C2E5F58363A201DFA3
:10285700EC75A20022E583C2E3F583E0A363A2013E
:10286700F0A363A201DFEE75A20022E583C2E4D2E2
:0A287700E3F583E0A363A201F0A3E0
:1028810063A201DFEC75A20022E58344F8F583E041
:10289100A363A201F0A363A201DFEE75A20022F9F6
:1028A10022C002C004C00612FFF0D006D004D0023C
:0128B1002204
:103ABF000A536572763A004572724C656E210A00A0
:103ACF00205544502054696D654750530A00200A11
:103ADF00444154414752414D3A20002043414E202A
:103AEF0054696D654750530A0020547261737353C4
:103AFF00656E644552520A000ACEF8C4EBE8EDFB3E
:103B0F0043414E210A000A45727241647243414E8D
:103B1F003A000A00205265496E69742043414E0AEB
:103B2F00002043414E283029203E20544F210A00C7
:0E3B3F0020545520300A0020545520310A0031
:03001E00E4FF22DA
:10436300C2A9438902758C48758A4875D90475DBDF
:104373004875DC4875DD4875DE48E4F5E9F5F9D2A2
:08438300D9C2DAD28CD2DE228D
:10433500C2D9907B17E07013E5E92419F5EB30D766
:1043450006E5F904F5FB2285F9FB22E5E924C8F524
:0E435500EB30D706E5F904F5FB2285F9FB22D3
:1041DB00C2D9907B17E0702C301D16E5E92432F51F
:1041EB00EB30D707E5F904F5FB800385F9FBC21D1E
:1041FB0022E5E92405F5EB30D706E5F904F5FB22BA
:10420B0085F9FB22E5E92432F5EB30D706E5F90415
:07421B00F5FB2285F9FB22EF
:10438B00124363907B17E0C394645006123F5412A0
:10439B004335120022D21CE4F557907C2FF0F546E2
:0743AB00F55BC21DF559226C
:10422200EF24FCF546200B127E3A7FBF1232A37EAA
:10423200777FF0E4FBAD46123594E546D3940D400A
:1042420010200B077E3A7FC61232A3E4F546D21A3B
:10425200229077F063A201907C1F63A201AF461205
:0542620027A4C21A228E
:0F447A00D3EF6480948D5006E55B70028F5B2258
:101F220020D903021FFF201C03021FFFE55B605242
:101F3200907478540FFF7D4812279BE54864017026
:101F42001E907480E0B4FF0ED21E200B127E3A7FE8
:101F5200CF1232A38009301E06E4F55B021FFF1286
:101F6200433512401C200B077E3A7FDD1232A3203C
:101F72000B0B7E747F78E4FBAD5B123594E4F55B6A
:101F8200807BE5466043907C23E02405F526D394CC
:101F92000D4007E4F546D21A8063907C1FE5265473
:101FA2000FFF7D4812279BE54830E702D21DE54826
:101FB200B40109301E06E54B6401600312401C1295
:101FC2004335E4F546D21A8034E558601E907B030F
:101FD200540FFF7D4812279BE548B40103201E03DE
:101FE20012401C124335E4F5588012201F0C907BDE
:101FF20017E0C39464500312407E124335122F0E31
:102002008F26EF70030220C61241DBE4F559E54842
:10201200B4010CD21E200B077E3A7FEA1232A3E5EE
:102022005AC394C8502D30032AE548B4420DE54BFB
:10203200B4020890772AE0640160187418255AF5F2
:1020420082E4347BF583E526255AF55A7D48AF268E
:10205200122792300121E54820E71C9079EF7D4854
:10206200AF26122792AF26123838EF700A200B07DC
:102072007E3A7FF81232A3E54854817047E526D3B1
:10208200940D400C200B3D7E3B7F071232A380341F
:10209200E54AD394074028200B2A7E3B7F15123253
:1020A200A390757B7D48AF261227927E757F7BE4D5
:1020B200FBAD261235947E3B7F211232A38005AF01
:1020C2002612376E300E2030001B907B17E0C3942F
:1020D2006450120559E55994F0400A9080007480CA
:1020E200F0C2AF80FEC20E2002030221E1E557607A
:1020F20031D39401400415578028907C2FE004F0DE
:10210200E0D39403400D200B077E3B7F231232A3C2
:1021120012438B200B077E3B7F301232A3E4F5572C
:10212200D21C301B43E558703F907B0304F0A3742C
:1021320008F0A37480F0A37401F0A37406F0907CFD
:102142001AE0907B08F0907C1BE0907B09F0907C79
:102152001CE0907B0AF0907C1DE0907B0BF0E4A3E6
:10216200F0A3F075580BC21B301972907C18E07006
:1021720035E5587031907B037442F0A37408F090F7
:102182007C19E0907B05F0907C1EE0907B06F0A32A
:102192007401F0755806200B077E3B7F3F1232A375
:1021A200907C18E004F0907C18E06402702FE558EF
:1021B200702B907B037402F0A37408F0907C19E0FA
:1021C200907B05F0A3F0A37401F0755806200B076D
:1021D2007E3B7F461232A3907C18E004F0C20212CA
:0421E200247AC20099
:0121E60022D6
:1042D300E55A602CE49078ECF0A3E55AF0907AF07C
:1042E300E09078EEF0A37419F0907B1863A201902C
:1042F30078F063A201AF5A1227A4E4F55A7F012292
:034303007F002216
:0B448900301A05C21A7F01227F0022BA
:0100210022BC
:0644AE00E4F55AF5462278
:0A449400E490757BF0A3F0A3F02282
:104306002043616E457247495400200A0045727287
:104316004C656E43616E21000A002043616E457252
:0F43260072434821000A205265714572722100CE
:102F0E00E59B541F6020200B1A7E437F061232A3CE
:102F1E00E59B541FFF7E007D031233A47E437F107A
:102F2E001232A3E4F59BE5BA30E010E4F5B375B1C7
:102F3E0080F5B2D21CF557907C2FF0E5CFF47003DC
:102F4E00023063752801E4F527E5CFF455287003A8
:102F5E00023051E527C454F0F5B1E5B2547F642038
:102F6E006003023022E5B3540FF54C85BC48E5BD35
:102F7E00541FFF131313541FFFE5BD54E044184FA5
:102F8E00F549E5BDC43354E0FFE5BE131313541FDA
:102F9E004FF54AE5BEC43354E0FFE5BF1313135497
:102FAE001F4FF54B85A34D85A34E85A34F85A3508B
:102FBE0085A35185A35285A35385A354E4F5B2206E
:102FCE001F0CE548547EB5480575B350800375B3A4
:102FDE00D0E54C700AE548547EB548037F00223098
:102FEE001F08E54830E7037F0022E54CD3940840E4
:102FFE001D200B177E437F131232A3AF4C7E007D34
:10300E00031233A47E437F1E1232A37F0022E54CAF
:10301E002405FF22E5B2549F6023200B207E437FC0
:10302E00201232A3AFB27E007D031233A4AFB37E63
:10303E00007D031233A47E437F1E1232A3E4F5B249
:10304E0075B3D0E52825E0F5280527E527C39408B4
:07305E005003022F577F0011
:013065002248
:10401C00907B17E0C39464505675B180E4F5B3F50A
:10402C00B28548BCE54AC4135407FFE54954E04F38
:10403C00F5BDE54A33333354F8FFE54BC41354074D
:10404C004FF5BEE54B33333354F8F5BF854DA3859F
:10405C004EA3854FA38550A38551A38552A38553A9
:10406C00A38554A3E54C540F2450F5B375570AC2DD
:02407C001C2204
:10407E0075B190E5B220E613200B107E437F2B1214
:10408E0032A3AFB27E007D031233A4E4F5B3F5B2D2
:10409E007471250FF582E43461F583E0F5BCE4F527
:1040AE00BD7472250FF582E43461F583E0FF33337E
:1040BE003354F8F5BE75BF78050F050F7471250FD3
:1040CE00F582E43461F583E07002F50F75B350228A
:09449E00EF6003C29622D29622BF
:103F540043AB01C2E8C2EAE4FFEFC454F0F5B1C3D5
:103F6400EF64809488500575B3D08003E4F5B3E41E
:103F7400F5B2F5BCF5BDF5BEF5BFF5C4F5C5F5C69E
:103F8400F5C7F5A3F5A3F5A3F5A3F5A3F5A3F5A349
:103F9400F5A30FBF0EC3907B17E0FF25E0F5B475C2
:103FA400B50C75B66C75A11275AB0275C13E75C3BF
:043FB400FF75C203D0
:013FB80022E6
:100EC9003E2A2C312CCFE0F0E0ECE5F2F0FB20F3E8
:100ED900EFF0E0E2EBFFFEF9E5E3EE20EAEEEDF2FA
:100EE900F0EEEBEBE5F0E020CACF20C8F1E5F2FC2B
:100EF9000A003E4C2C6B30312C25732C43EAEEF062
:100F0900EEF1F2FC20EDE020F8E8EDE52043414E5A
:100F19002C30202D20353030EAE1283530EC292CD1
:100F290031202D203530EAE128353030EC290A000E
:100F390030202D20353030EAE1283530EC290031D8
:100F4900202D203530EAE128353030EC29003E5398
:100F59002C6B30322C2562752CCCE0EAF12E20E086
:100F6900E4F0E5F120E1EBEEEAE020D2D128302DE2
:100F790038290A003E532C6B30332C2562752CCC52
:100F8900E0EAF12E20E0E4F0E5F120E1EBEEEAE021
:100F990020D2C8D228302D38290A003E532C6B3074
:100FA900342C2562752CCCE0EAF12E20E0E4F0E542
:100FB900F120E1EBEEEAE020D2D328302D38290ADE
:100FC900003E422C6330312C2562752CC2F2EEF0C2
:100FD900E8F7EDFBE920EAEEEDF2F0EEEBEBE5F0F8
:100FE90020EDE020F8E8EDE50A003E2A2C312CCF6F
:100FF900F0EEF2EEEAEEEB20C8F1E5F2FC2DCCE0E2
:10100900E3E8F1F2F0E0EBFCEDFBE920EDE020EFA5
:10101900EEF0F2F32052533233320A003E4C2C6B7D
:1010290030352C256C752CD1EAEEF0EEF1F2FC206E
:10103900EEE1ECE5EDE020EDE020EFEEF0F2F32C4F
:101049003130302C3230302C3330302C3630302C9B
:10105900313230302C323430302C343830302C3975
:101069003630302C31393230302C33383430302C62
:1010790035373630302C3131353230300A003E5375
:101089002C6B30362C2562752CC0E4F0E5F120CAB2
:10109900CF20E4EBFF20ECE0E3E8F1F2F0E0EBE84D
:1010A9000A003E532C6B31322C2562752CCAEEEBAB
:1010B9002DE2EE20E1EBEEEAEEE220E220EEF2E2B2
:1010C900E5F2E52028EFE0EAE5F23D352B6E2A311D
:1010D9003320E1E0E9F2290A003E532C6B31332C2D
:1010E9002562752CC7E0E4E5F0E6EAE020F1F2E0DC
:1010F900F0F2E020EFE5F0E5E4E0F7E828ECF1298B
:101109000A003E422C6B30392C2562752CCDE52026
:10111900EFE5F0E5E4E0E2E0F2FC20E4E8E0E3ED0D
:10112900EEF1F2E8EAF30A003E422C6B31302C254D
:1011390062752CCFE5F0E5E7E0E3F0F3E7EAE020BC
:10114900EFF0E820EEF2F1F3F2F1F2E2E8E820EE56
:10115900E1ECE5EDE0203220ECE8ED2E0A003C213F
:10116900003C6B30313D003C6B30323D003C6B3014
:10117900333D003C6B30343D003C6330313D003C35
:101189006B30353D003C6B30363D003C6B31333DB7
:10119900003C6B30393D003C6B31303D00CEF820CE
:1011A900E4EBE8EDFB210A000A4173796E634F55C0
:1011B900543A000A435243204552523A20000A4108
:1011C90073796E63494E3A00CFE0EAE5F220E220F6
:1011D90043414E0A00D2D320320A00D2D320330A27
:1011E90000C0F0F5D2D10A003F3F3F0A0000891242
:1011F9009B24AD36BF48C15AD36CE57EF78108936D
:101209001AA52CB73EC940DB52ED64FF76028B105C
:101219009926AF34BD4AC358D16EE77CF5830A914C
:1012290018A72EB53CCB42D950EF66FD74048D1634
:101239009F20A932BB4CC55ED768E17AF3850C972C
:101249001EA128B33ACD44DF56E960FB72068F141C
:101259009D22AB30B94EC75CD56AE378F1870E950C
:101269001CA32AB138CF46DD54EB62F97008811A04
:10127900932CA53EB740C952DB64ED76FF89009BEC
:1012890012AD24BF36C148D35AE56CF77E0A8318DC
:10129900912EA73CB542CB50D966EF74FD8B0299CC
:1012A90010AF26BD34C34AD158E76EF57C0C851EB4
:1012B9009728A13AB344CD56DF60E972FB8D049FAC
:1012C90016A920BB32C54CD75EE168F37A0E871C9C
:1012D900952AA338B146CF54DD62EB70F98F069D8C
:1012E90014AB22B930C74ED55CE36AF178001123FB
:1012F90032465765748C9DAFBECADBE9F8100133DD
:1013090022564775649C8DBFAEDACBF9E8213002CD
:101319001367764455ADBC8E9FEBFAC8D9312012BC
:101329000377665445BDAC9E8FFBEAD8C942536129
:101339007004152736CEDFEDFC8899ABBA5243719C
:101349006014053726DECFFDEC9889BBAA6372408D
:101359005125340617EFFECCDDA9B88A9B7362507C
:101369004135241607FFEEDCCDB9A89A8B8495A7E1
:10137900B6C2D3E1F008192B3A4E5F6D7C9485B75C
:10138900A6D2C3F1E018093B2A5E4F7D6CA5B4864D
:1013990097E3F2C0D129380A1B6F7E4C5DB5A4963C
:1013A90087F3E2D0C139281A0B7F6E5C4DC6D7E5A9
:1013B900F48091A3B24A5B69780C1D2F3ED6C7F51C
:1013C900E49081B3A25A4B79681C0D3F2EE7F6C40D
:1013D900D5A1B082936B7A48592D3C0E1FF7E6D4FC
:0D13E900C5B1A092837B6A58493D2C1E0FB0
:030023000238E2BE
:0D38E200C0E0C0F0C083C082C0D075D01817
:1038EF0030985AC298750B01AF99202013BF550914
:1038FF00756300D220D2918044906F30EFF0803DFD
:10390F00E56D703474322563F582E4346FF583EF1F
:10391F00F0E563B40104EF04F55FE563600AB55F9A
:10392F001304F56DC291800CEF64556007C22090AF
:10393F006F30EFF005638005906F30EFF03099290D
:10394F00302124D290E56AB5620DC221D223C290F4
:10395F00E4FF12449E80107432256AF582E43470BD
:09396F00F583E0F599056AC2999F
:0B397800D0D0D082D083D0F0D0E0325D
:10349E007BFF7A0E79C9121961907B17E070147553
:1034AE002EFF752F0F7530397BFF7A0E79FB1219AF
:1034BE00618012752EFF752F0F7530487BFF7A0EC7
:1034CE0079FB1219617BFF7A0F7957906170E0F5E5
:1034DE002E1219617BFF7A0F797D90616BE0F52ECC
:1034EE001219617BFF7A0F79A4906102E0F52E121A
:1034FE0019617BFF7A0F79CAA21FE433F52E1219D8
:10350E00617BFF7A0F79F3121961907472E0FEA35A
:10351E00E0FFC3E49FFFE49EFEAB07FA3395E0F9AC
:10352E00F87F007E8C7D0A7C001222398F318E301E
:10353E008D2F8C2E7BFF7A1079251219617BFF7AE5
:10354E00107987856C2E1219617BFF7A1079AB90FA
:10355E006F2EE0F52E1219617BFF7A1079E29061E1
:10356E006EE0F52E1219617BFF7A11790BA222E41F
:10357E0033F52E1219617BFF7A117931906F31E09C
:06358E00F52E1219612266
:103066007E117F67123BD9EF4E70037F0122E490F9
:103076007B17F07E117F6A123BD9EF4E6015124422
:1030860033BF3106907B17740AF0BF3206907B1768
:103096007464F09061027402F090616BF09061705C
:1030A600F07E117F70123BD9EF4E60081240DE9021
:1030B6006170EFF07E117F76123BD9EF4E600812F9
:1030C60040DE90616BEFF07E117F7C123BD9EF4EB4
:1030D60060081240DE906102EFF07E117F82123BA3
:1030E600D9EF4E600D1240DEEC4D4E4F24FF921F7D
:1030F6008002C21F7E117F88123BD9EF4E602312D9
:1031060040DEA804A905AA06AB077F007E8C7D0ACF
:103116007C001222391222CB907472EEF0A3EFF0EB
:10312600800A90747274FFF0A374B8F07E117F8EDB
:10313600123BD9EF4E60071240DE8F6C8003756C30
:1031460001906F2E7401F07E117F94123BD9EF4EE1
:10315600600A1240DE90616EEFF08005E490616EC9
:10316600F07E117F9A123BD9EF4E600C124433EF7A
:1031760024D024FF92228002D2227E117FA0123B0D
:10318600D9EF4E600C124433EF24D0906F31F080AB
:0831960005E4906F31F07F00A9
:01319E00220E
:1028B200C221C223C220E4906F2FF0F56AF562F5BF
:1028C200089061A4F0F563F50B90747274FFF0A3A5
:1028D20074F4F0123066E4F50F907C417461F0A359
:1028E2007471F0906170E0F50FE50FC39401400739
:1028F200E50FD394084003E4F50FE50F6028907CC0
:1029020041E475F0011221E785F082F58374C4F089
:10291200150F907C41E475F0011221E785F082F5F4
:1029220083E50FF080D490616BE0F50FE50FC3945F
:10293200014007E50FD394084003E4F50FE50F606B
:1029420028907C41E475F0011221E785F082F5833D
:1029520074C8F0150F907C41E475F0011221E785EF
:10296200F082F583E50FF080D4906102E0F50FE587
:102972000FC394014007E50FD394084003E4F50F19
:10298200E50F6028907C41E475F0011221E785F0A3
:1029920082F58374C2F0150F907C41E475F0011248
:1029A20021E785F082F583E50FF080D4907C41E445
:1029B20075F0011221E785F082F583E4F0907C4105
:1029C20075F0011221E785F082F583E4F0F50FF549
:1029D2006BE4F55D75F075E56BA42453F582E5F0C3
:1029E2003468F58375F00DE55D122327E4F0055D8B
:1029F200E55DB408DF75F075E56BA42446F582E564
:102A0200F03468F583E4F0E56B75F00DA42403F56A
:102A120082E43461F583E4F0F56175F068E56BA456
:102A22002432F582E5F03471F58375F00DE561121B
:102A32002327E4F00561E561B408DF056BE56B640B
:102A420008708EE4F571F55CF55EF560F569F56E7A
:102A5200F561F55DF56BF568C2ADF5C9D2CDD2CCA5
:102A6200C2C9C2CAF5CDF5CC907472E0F5CBA3E031
:102A7200F5CA85CBCD85CACCD29ED29CD2CAC2AC75
:0C2A8200C298C29975B81075B710D2AC9C
:012A8E002225
:0100220022BB
:10376E008F2730220EE548B44209E54B6402700300
:10377E00023837E54954E324DF604A24DF60291418
:10378E00602624E3605C24E0601E2460600302383F
:10379E0037E54A75F00DA42403F582E43461F58310
:1037AE007D48AF271227922275F00DE560A424EE16
:1037BE00F582E5F0346BF5837D48AF27122792052D
:1037CE006053603F2275F00DE55CA424C5F582E5DB
:1037DE00F03461F5837D48AF27122792055C535C68
:1037EE007F2275F075E54AA42453F582E5F034681E
:1037FE00F583E54B543FFF1313543F75F00D122321
:10380E00277D48AF2712279275F068E54AA4243227
:10381E00F582E5F03471F583E54B543FFF131354F5
:0A382E003F75F00D122327E4F0228D
:101C5B00E4F528906F2EE0FFE528C39F4003021E9A
:101C6B0073E560655E605A75F00DE55EA424F2F5D0
:101C7B0082E5F0346BF583E02405F529C3940E500F
:101C8B002E75F00DE55EA424EEF582E5F0346BF5D0
:101C9B008363A20174022568F582E43460F58363E3
:101CAB00A201AF291227A4E5292568F568800A202F
:101CBB000B077E117FA61232A3055E535E3F021EF9
:101CCB006E75F075E56BA42453F582E5F03468F579
:101CDB008375F00DE55D122327E07003021D8F75F0
:101CEB00F075E56BA42457F582E5F03468F5837540
:101CFB00F00DE55D122327E02405F529C3940E5062
:101D0B003675F075E56BA42453F582E5F03468F570
:101D1B008375F00DE55D12232763A201740225681C
:101D2B00F582E43460F58363A201AF291227A4E5A1
:101D3B00292568F568800A200B077E117FA61232D1
:101D4B00A375F075E56BA42453F582E5F03468F5C3
:101D5B008375F00DE55D122327E4F0055DE55DC3AA
:101D6B0094085003021E6EE4F55D75F075E56BA4E7
:101D7B002446F582E5F03468F583E4F0056B536B8C
:101D8B0007021E6EE55C6571605A75F00DE571A476
:101D9B0024C9F582E5F03461F583E02405F529C308
:101DAB00940E502E75F00DE571A424C5F582E5F067
:101DBB003461F58363A20174022568F582E4346013
:101DCB00F58363A201AF291227A4E5292568F568DD
:101DDB00800A200B077E117FA61232A30571537167
:101DEB007F021E6EE56975F00DA42403F582E434C1
:101DFB0061F583E06068E56975F00DA42407F58251
:101E0B00E43461F583E02405F529C3940E502DE5E8
:101E1B006975F00DA42403F582E43461F58363A2A4
:101E2B000174022568F582E43460F58363A201AF87
:101E3B00291227A4E5292568F568800A200B077E5F
:101E4B00117FA61232A3E56975F00DA42403F58268
:101E5B00E43461F583E4F00569536907800505698E
:101E6B005369070528021C5E856829E4F5689070A4
:101E7B00327455F0A3F0E5292405A3F0E4A3F0A3F5
:101E8B00E56CF0906845E0907037F0E529601190B3
:101E9B00600263A20190703863A201AF291227A4DC
:101EAB00E4F564F565E5292403F56790703563A2C5
:101EBB00019011F663A201AF67AE66AD65AC64121B
:101ECB0027E08F678E668D658C6474382529F582C3
:101EDB00E43470F583E565F074392529F582E43433
:101EEB0070F583E564F0E5292408F562D221E4F569
:101EFB006A90616FF07F0112449EC2992099FDD2C6
:101F0B0099200B127E117FB11232A37E707F32E4C7
:061F1B00FBAD62123594DB
:011F2100229D
:10247A00E56975F00DA42403F582E43461F583E07F
:10248A007005056953690775F075E56BA42453F562
:10249A0082E5F03468F58375F00DE55D122327E0D7
:1024AA007023055DE55DC39408401AE4F55D75F097
:1024BA0075E56BA42446F582E5F03468F583E4F00B
:1024CA00056B536B07300020C200906F31E0601239
:1024DA0004F0E0D394F0400A9080007480F0C2AF18
:1024EA0080FE90616FE004F030DA3FC2DA9061A4B6
:1024FA00E0FF906F2FE0FDC39F502FE57025ECF5AC
:10250A00EC30D709E56F25FC04F5FC8006E56F255C
:10251A00FCF5FC74A52DF582E43461F583E0B56C15
:10252A0003121C5B906F2FE004F030210F90616F53
:10253A00E0D39414400BC221D2238005E490616F4A
:10254A00F0906F30E0FF600C7E007D031233A4E44C
:10255A00906F30F0E56D70030226C8F527E4F56444
:10256A00F565E52724FEF567906F3463A2019011A3
:10257A00F663A201AF67AE66AD65AC641227E08F61
:10258A00678E668D658C64C220E4F56DE5654564E9
:10259A006022300B030226C87E117FBC1232A37E52
:1025AA006F7F32E4FBAD271235947D03AF65AE64CD
:1025BA001233A422200B127E117FC71232A37E6F20
:1025CA007F32E4FBAD27123594906F34E0FB64014F
:1025DA006003022663906F36E09061A3F06007E023
:1025EA0020E7030226C89061A3E0547FF090684573
:1025FA00F0E5E92402F5EC30D707E5F904F5FC80AB
:10260A000385F9FCC2DA906F35E075F064A485F0B1
:10261A006FF570906F37E0FE541F9061A4F0EEC41E
:10262A0013540704906F2EF0E4A3F0F5279061A4E9
:10263A00E0FFE527C39F40030226C874382527F523
:10264A0082E4346FF583E0FF74A52527F582E4342C
:10265A0061F583EFF0052780D4906F35E0656C70E3
:10266A005DEB24FD602D14603514603D2403704435
:10267A00200B077E117FD11232A3E558704075589E
:10268A000D906F3763A201907B0363A201AF5812CA
:10269A0027A422200B287E117FDE1232A322200BD0
:1026AA001D7E117FE41232A322200B127E117FEAD3
:0E26BA001232A322200B077E117FF11232A3F1
:0126C80022EF
:103B59000208A4E493A3F8E493A34003F68001F2D6
:103B690008DFF48029E493A3F85407240CC8C3336D
:103B7900C4540F4420C8834004F456800146F6DF3C
:103B8900E4800B01020408102040809044A7E47EE1
:103B9900019360BCA3FF543F30E509541FFEE49331
:103BA900A360010ECF54C025E060A840B8E493A3F8
:103BB900FAE493A3F8E493A3C8C582C8CAC583CA23
:103BC900F0A3C8C582C8CAC583CADFE9DEE780BEDB
:0144AD00000E
:1021E700A3F8E0C5F025F0F0E582158270021583AB
:0621F700E0C838F0E82208
:1021FD0075F008758200EF2FFFEE33FECD33CDCC99
:10220D0033CCC58233C5829BED9AEC99E58298401B
:10221D000CF582EE9BFEED9AFDEC99FC0FD5F0D6F8
:10222D00E4CEFBE4CDFAE4CCF9A88222B800C1B922
:10223D000059BA002DEC8BF084CFCECDFCE5F0CB60
:10224D00F97818EF2FFFEE33FEED33FDEC33FCEB99
:10225D0033FB10D703994004EB99FB0FD8E5E4F954
:10226D00FA227818EF2FFFEE33FEED33FDEC33FC41
:10227D00C933C910D7059BE99A4007EC9BFCE99A35
:10228D00F90FD8E0E4C9FAE4CCFB2275F010EF2F7A
:10229D00FFEE33FEED33FDCC33CCC833C810D7077A
:1022AD009BEC9AE899400AED9BFDEC9AFCE899F8B5
:0E22BD000FD5F0DAE4CDFBE4CCFAE4C8F92248
:0E22CB00C3E49FFFE49EFEE49DFDE49CFC2224
:1022D900EB9FF5F0EA9E42F0E99D42F0E89C45F05B
:0122E90022D2
:0C22EA00ECF0A3EDF0A3EEF0A3EFF02267
:1022F600A8828583F0D083D08212230D12230D127B
:10230600230D12230DE473E493A3C583C5F0C5839F
:10231600C8C582C8F0A3C583C5F0C583C8C582C831
:012326002294
:0C232700A42582F582E5F03583F58322C1
:1018FF00E53A242EF8E6053A22782B301702782E97
:10190F00E475F0011223DA0223332010EB7F2ED27D
:10191F00108018EF540F2490D43440D4FF30140BA0
:10192F00EF24BFB41A0050032461FFE53B6002159A
:10193F003B053EE53E7002053D30170D782BE475F3
:10194F00F0011223DAEF0223790241947403D217C4
:10195F008003E4C217F53A8B2B8A2C892DE4F53BD3
:10196F00F53DF53EE53B60077F2012193A80F5758E
:10197F003CFFC211C210C212C213C215C216C21846
:10198F00121908FF700D3017057F0012194BAF3E6B
:10199F00AE3D22B4255FC2D5C214121908FF24D060
:1019AF00B40A00501A75F00A783B30D50508B6FF17
:1019BF000106C6A426F620D5047002D21380D924BE
:1019CF00CFB41A00EF5004C2E5D214021B4BD21150
:1019DF0080C6D21080C0D21280BCD2D580BAD215A8
:1019EF0080B47F2012193A2012077401B53B0040D2
:1019FF00F11218FFFF12193A021973D218D216807A
:101A0F00951218FFFB1218FFFA1218FFF94A4B70C4
:101A1F0006791C7A1C7BFF20122EE53B602A7E0084
:101A2F008E8275830012234C60060EEE653C70F0BB
:101A3F00C2D5EBC0E0EAC0E0E9C0E0EE121B92D0E5
:101A4F00E0F9D0E0FAD0E0FB122333FF60AAEBC03D
:101A5F00E0EAC0E0E9C0E012193AD0E02401F9D081
:101A6F00E03400FAD0E0FBE53C0460DCD53CD980E3
:101A7F00877BFF7A1B798ED212809C791080027936
:101A8F0008C216C2188008D2D5790A8004790AC212
:101A9F00D5E53C047002F53CE4FAFDFEFF1218FF99
:101AAF00FC7B082011131218FFFD7B1030100A1257
:101ABF0018FFFE1218FFFF7B20EC3382D592D55012
:101ACF0013C3E43010069FFFE49EFEE42011039D34
:101ADF00FDE49CFCE4CBF8C211EC700CCFCECDCC66
:101AEF00E824F8F870F38017C3EF33FFEE33FEED01
:101AFF0033FDEC33FCEB33FB994002FB0FD8E9EBE2
:101B0F00301105F8D0E0C448B211C0E00AEC4D4ED8
:101B1F004F78207B0070C2EAB53C0040BCC0E01299
:101B2F001B94D0F0D0E0201104C4C0E0C4B211C0A7
:101B3F00F0121923D0F0D5F0EB0219731224391AD1
:101B4F0010531A8A5819E14C19DD421A8E4F1A9602
:0F1B5F00441A964919F6431A9C551A80461A8063
:101B6E00451A80471C3C5019E52D19E92E1A0C2BED
:101B7E0019ED231A0A201C252A19A54800001A045B
:101B8E003F3F3F00790AA2D5201314301509B91032
:101B9E00020404B9080104A2D52016025001042043
:101BAE0012689212B53B005034C0E07F20301319FA
:101BBE007F30A21272167215500F121BEBC212C298
:101BCE0016C215C2187F30800F301503E9C0E0121F
:101BDE00193A301503D0E0F9D0E0B53BCC301517EB
:101BEE007F30B9100C12193A7F583014077F788065
:101BFE0003B9080312193A3012057F2D02193A7FE4
:101C0E00202018F87F2B2016F322921280CF286EF8
:101C1E00756C6C2900D2111218FF3011F8C21178B0
:101C2E003B30D50108F60219A52D5043495812181C
:101C3E00FF2403B405004001E4901C379312192BC6
:0D1C4E00743A12192BD213753B04021A8A46
:102A8F008B2B8A2C892DE4F537F536F535F534F592
:102A9F0032F533E52F4530452E6012EBC0E0EAC02A
:102AAF00E0E9C0E0AB2EAA2FA9301223EAAB2B0529
:102ABF002DE52DAA2C7002052C14F9122333F538AD
:102ACF00C394094007E538D3940D40E1E5386420FD
:102ADF0060DBE538B42D054333038016E538B42B9E
:102AEF0005433301800C74FF252DF52D74FF352C14
:102AFF00F52CE53160046410703FAB2BAA2CA92D87
:102B0F0012233364306009E531702E75310A802944
:102B1F0090000112234CFF64786004EFB458134304
:102B2F0033017531107402252DF52DE4352CF52C5C
:102B3F008007E5317003753108AB2B052DE52DAA04
:102B4F002C7002052C14F9122333F538C39461400D
:102B5F000AE538D3947A50035338DF74D02538F50B
:102B6F0038C3940A400CE5389411406D74F9253838
:102B7F00F538E538D39531506043330185373C85BF
:102B8F00363B85353A853439AF317E00E4FCFDABF9
:102B9F0037AA36A935A83412238BC8ECC8C9EDC99A
:102BAF00CAEECACBEFCBE4FCFDFEEB2538F537EED2
:102BBF003AF536ED39F535EC38F534AF37AE36AD8D
:102BCF0035FCAB3CAA3BA93AA839D31222D9500302
:102BDF00022B48433304022B48E53320E003E48003
:102BEF002DE52F4530452E601EAB2BE52D24FFF92B
:102BFF00E52C34FFFAEBC0E0EAC0E0E9C0E0AB2E11
:102C0F00AA2FA9301223EAE53330E20774FFFFFE43
:102C1F00FDFC22E533AF37AE36AD35AC3430E103D2
:042C2F000222CB2290
:10233300BB010689828A83E0225002E722BBFE02A8
:09234300E32289828A83E49322DB
:10234C00BB010CE58229F582E5833AF583E0225046
:10235C0006E92582F8E622BBFE06E92582F8E22290
:0D236C00E58229F582E5833AF583E49322AA
:10237900BB010689828A83F0225002F722BBFE0143
:02238900F3223D
:10238B00E88FF0A4CC8BF0A42CFCE98EF0A42CFCF1
:10239B008AF0EDA42CFCEA8EF0A4CDA8F08BF0A46F
:1023AB002DCC3825F0FDE98FF0A42CCD35F0FCEBCE
:1023BB008EF0A4FEA9F0EB8FF0A4CFC5F02ECD3993
:0F23CB00FEE43CFCEAA42DCE35F0FDE43CFC2200
:1023DA00FAE6FB0808E6F925F0F618E6CA3AF62204
:1023EA00BB011A89828A83D0F0D0E0F8D0E0F9D014
:1023FA00E0FAD0E0FBE8C0E0C0F00224685016E939
:10240A00F8D083D082D0E0F9D0E0FAD0E0FBC082E5
:10241A00C08302245FBBFE16E9F8D083D082D0E0E5
:0F242A00F9D0E0FAD0E0FBC082C0830224712217
:10243900D083D082F8E4937012740193700DA3A332
:1024490093F8740193F5828883E473740293686046
:06245900EFA3A3A380DF46
:09245F00EBF608EAF608E9F622A2
:09246800EBF0A3EAF0A3E9F02275
:09247100EBF208EAF208E9F2229C
:00000001FF
